:100000000C9434000C943E000C943E000C943E0082
:100010000C943E000C943E000C943E000C943E0068
:100020000C943E000C943E000C943E000C943E0058
:100030000C943E000C943E000C943E000C943E0048
:100040000C943E000C943E000C943E000C943E0038
:100050000C943E000C943E000C943E000C943E0028
:100060000C943E000C943E0011241FBECFEFD4E050
:10007000DEBFCDBF0E9440000C946F040C940000C2
:100080007F928F929F92AF92BF92CF92DF92EF9228
:10009000FF920F931F93CF93DF935298539A3C98FC
:1000A000449A3D98459A84B18F6384B98AB1806C33
:1000B0008AB987B1837C87B988B18C6388B98AB1E2
:1000C0008F7C8AB98BB180638BB93898409880E86F
:1000D00080937A0080E280937C0080917A00876030
:1000E00080937A0080917A00806480937A0030E077
:1000F00020E0772406C030E021E010E00DC031E0C0
:1001000020E088249924AA24BB24DD24EE24FF24A3
:1001100000E0F3CF31E020E080917A0084FFFCCF53
:1001200080917A00806180937A009091790080912B
:100130007A00806480937A0086B18C7039F4492FFC
:1001400042954695477097E0C92E17C0883039F41C
:10015000492F42954F70485F8FE0C82E0EC096958C
:1001600096959695843029F4492F405FBFE1CB2EB8
:1001700004C0492F405EAFE3CA2E319902C07724F4
:100180000FC0772019F0772473940AC077247394F2
:100190009924AA24BB24DD24EE24FF2400E010E0EF
:1001A0004A9B1DC2332309F0B6CF5B983499EFC048
:1001B000992009F42898AA2009F42998BB2009F469
:1001C0002A98DD2009F42B98EE2009F42C98FF20C2
:1001D00009F42D98002309F45F98112309F45E981F
:1001E0008C2D842335997EC0292D30E0869590E0B2
:1001F00001962817390709F4289AE42FF0E0CC2D4E
:10020000D0E02A2D30E0CF0101968C239D2362E0BF
:1002100070E00E9448046F5F7F4F2617370709F48C
:10022000299A2B2D30E0CF0102968C239D2362E08A
:1002300070E00E9448046F5F7F4F2617370709F46C
:100240002A9A2D2D30E0CF0103968C239D2362E066
:1002500070E00E9448046F5F7F4F2617370709F44C
:100260002B9A2E2D30E0CF0104968C239D2362E043
:1002700070E00E9448046F5F7F4F2617370709F42C
:100280002C9A2F2D30E0CF0105968C239D2362E020
:1002900070E00E9448046F5F7F4F2617370709F40C
:1002A0002D9A202F30E0CF0106968C239D2362E00B
:1002B00070E00E9448046F5F7F4F2617370709F4EC
:1002C0005F9A212F30E03796CF018C239D2362E087
:1002D00070E00E9448046F5F7F4F2617370709F0D0
:1002E0004DC1EEC09394891508F49924A39450E06D
:1002F0006C2D70E02A2D30E0CA01019686239723E9
:10030000821793070CF4AA24B3942B2D30E0CA0172
:10031000029686239723821793070CF4BB24D39469
:100320002D2D30E0CA010396862397238217930769
:100330000CF4DD24E3942E2D30E0CA0104968623CC
:100340009723821793070CF4EE24F3942F2D30E0BB
:10035000CA01059686239723821793070CF4FF247E
:100360000F5F202F30E0CA0106968623972382175D
:1003700093070CF400E01F5F812F90E0495F5F4F0F
:1003800046235723481759070CF0F8C0F6C08C2DA8
:100390008423359997C0292D30E0869590E0019609
:1003A0002817390709F42898E42FF0E0CC2DD0E085
:1003B0002A2D30E0CF0101968C239D2362E070E06E
:1003C0000E9448046F5F7F4F2617370709F429986A
:1003D0002B2D30E0CF0102968C239D2362E070E04C
:1003E0000E9448046F5F7F4F2617370709F42A9849
:1003F0002D2D30E0CF0103968C239D2362E070E029
:100400000E9448046F5F7F4F2617370709F42B9827
:100410002E2D30E0CF0104968C239D2362E070E006
:100420000E9448046F5F7F4F2617370709F42C9806
:100430002F2D30E0CF0105968C239D2362E070E0E4
:100440000E9448046F5F7F4F2617370709F42D98E5
:10045000202F30E0CF0106968C239D2362E070E0D0
:100460000E9448046F5F7F4F2617370709F45F9893
:10047000212F30E03796CF018C239D2362E070E07E
:100480000E9448046F5F7F4F2617370709F45E9874
:10049000992009F4289AAA2009F4299ABB2009F482
:1004A0002A9ADD2009F42B9AEE2009F42C9AFF20D9
:1004B00009F42D9A002309F45F9A112309F05EC014
:1004C0005E9A5CC09394891510F428989924A3949B
:1004D00050E06C2D70E02A2D30E0CA010196862391
:1004E00097238217930714F42998AA24B3942B2DE9
:1004F00030E0CA010296862397238217930714F4EB
:100500002A98BB24D3942D2D30E0CA01039686236C
:1005100097238217930714F42B98DD24E3942E2D50
:1005200030E0CA010496862397238217930714F4B8
:100530002C98EE24F3942F2D30E0CA0105968623E3
:1005400097238217930714F42D98FF240F5F202F11
:1005500030E0CA010696862397238217930714F486
:100560005F9800E01F5F812F90E0495F5F4F462357
:1005700057234817590714F45E9810E04C991CC093
:100580002C2D30E0482D4F5F4D990AC0842E842FCA
:1005900090E02F5F3F4F220F331F220F331F07C002
:1005A000842E842F90E02F5F3F4F220F331F82173E
:1005B00093070CF0A4CDAECD4D99ACCD8394482DCE
:1005C00050E02C2D30E02F5F3F4FC901880F991F5D
:1005D000820F931F481759070CF091CD9BCD222312
:1005E00011F030E099CD5B9A359949C1292D30E061
:1005F0008C2D8423349977C090E00196959587954A
:100600002817390709F4289AE42FF0E0CC2DD0E020
:100610002A2D30E0CF0101968C239D23019662E0C4
:1006200070E00E9448042617370709F4299A2B2DF9
:1006300030E0CF0102968C239D23019662E070E0AA
:100640000E9448042617370709F42A9A2D2D30E016
:10065000CF0103968C239D23019662E070E00E94F7
:1006600048042617370709F42B9A2E2D30E0CF01C6
:1006700004968C239D23019662E070E00E9448045A
:100680002617370709F42C9A2F2D30E0CF01059655
:100690008C239D23019662E070E00E944804261797
:1006A000370709F42D9A202F30E0CF0106968C23CE
:1006B0009D23019662E070E00E94480426173707E8
:1006C00009F45F9A212F30E03796EC23FD23CF0108
:1006D000019662E070E00E9448042617370709F08F
:1006E00077C05E9A75C090E001969595879528171A
:1006F000390709F42898E42FF0E0CC2DD0E02A2D1A
:1007000030E0CF0101968C239D23019662E070E0DA
:100710000E9448042617370709F429982B2D30E04A
:10072000CF0102968C239D23019662E070E00E9427
:1007300048042617370709F42A982D2D30E0CF01F9
:1007400003968C239D23019662E070E00E9448048A
:100750002617370709F42B982E2D30E0CF01049689
:100760008C239D23019662E070E00E9448042617C6
:10077000370709F42C982F2D30E0CF0105968C23F4
:100780009D23019662E070E00E9448042617370717
:1007900009F42D98202F30E0CF0106968C239D235D
:1007A000019662E070E00E9448042617370709F4BA
:1007B0005F98212F30E03796EC23FD23CF0101967F
:1007C00062E070E00E9448042617370709F45E983B
:1007D00093948C2D8423891508F49924A39450E0D4
:1007E0006C2D70E02A2D30E0CA01019686239723F4
:1007F000821793070CF4AA24B3942B2D30E0CA017E
:10080000029686239723821793070CF4BB24D39474
:100810002D2D30E0CA010396862397238217930774
:100820000CF4DD24E3942E2D30E0CA0104968623D7
:100830009723821793070CF4EE24F3942F2D30E0C6
:10084000CA01059686239723821793070CF4FF2489
:100850000F5F202F30E0CA01069686239723821768
:1008600093070CF400E01F5F812F90E0495F5F4F1A
:1008700046235723481759070CF43DCC06C085B1D1
:100880008F6385B98BB1806C8BB930E021E044CCAB
:1008900097FB092E07260AD077FD04D00CD006D08E
:1008A00000201AF4709561957F4F0895F6F79095A2
:1008B00081959F4F0895AA1BBB1B51E107C0AA1F3A
:1008C000BB1FA617B70710F0A61BB70B881F991FF1
:1008D0005A95A9F780959095BC01CD010895F8949B
:0208E000FFCF48
:00000001FF
